:020000040001F9
:10900000C03D0020C1930100C9930100CB93010032
:10901000CD930100CF930100D19301000000000027
:10902000000000000000000000000000D3930100D9
:10903000D593010000000000D7930100D9930100EF
:1090400039970100DB930100099B0100DB930100CC
:10905000DB9301000000000071950100DB9301002B
:10906000DB930100DB930100DB930100DB93010044
:10907000DB930100DB930100DB930100DB93010034
:10908000DB93010091970100DB930100DB9301006A
:1090900015980100DB93010019980100DB93010092
:1090A000DB930100DB9301000000000000000000E2
:1090B000DB930100DB9301000000000000000000D2
:1090C00000000000000000000000000000000000A0
:1090D0000000000000000000000000000000000090
:1090E0000000000000000000000000000000000080
:1090F0000000000000000000000000000000000070
:10910000000000000000000000000000000000005F
:10911000000000000000000000000000000000004F
:10912000000000000000000000000000000000003F
:10913000000000000000000000000000000000002F
:10914000000000000000000000000000000000001F
:10915000000000000000000000000000000000000F
:1091600000000000000000000000000000000000FF
:1091700000000000000000000000000000000000EF
:1091800000000000000000000000000000000000DF
:1091900000000000000000000000000000000000CF
:1091A00000000000000000000000000000000000BF
:1091B00000000000000000000000000000000000AF
:1091C000000000000000000000000000000000009F
:1091D000000000000000000000000000000000008F
:1091E000000000000000000000000000000000007F
:1091F000000000000000000000000000000000006F
:10920000DFF80CD000F076F900480047E1BB010020
:10921000C03D002030B450E8012F93B2C4892344EC
:109220008489A34228BF1B1B0489A34202BFBFF34A
:109230002F8F002007E0C3EA020340E80134002C2E
:10924000E9D14FF001000A6030BC704750E8012FAF
:10925000C2EA024240E801210029F7D1704730B448
:1092600050E8022F1FFAA2F3C488A34202BFBFF343
:109270002F8F00200DE0C48923448489A34228BF96
:109280001B1BC2EA034340E80234002CE8D14FF034
:1092900001000A6030BC704750E8022FC2EA224247
:1092A00040E802210029F7D17047034653E8022F16
:1092B000D988B2EB324F4FF0000017BF92B241EAAB
:1092C000014142EA014104E05A68B2EB324F08BF63
:1092D000012043E80212002AE8D1704730B4044666
:1092E00054E8000F0D4644E80053002BF8D11560F8
:1092F00030BC704730B4044654E8000F40EA010522
:1093000044E80053002BF7D1156030BC704730B4EF
:10931000044654E8000F00EA010544E80053002B1E
:10932000F7D1156030BC704730B4044654E8000FE4
:1093300080EA010544E80053002BF7D1156030BCEA
:10934000704730B4044654E8000F00EB010544E8D0
:109350000053002BF7D1156030BC704730B4044681
:1093600054E8000FA0EB010544E80053002BF7D1AF
:10937000156030BC704770B404464FF0000054E8EC
:10938000006F0D68AE4207BF44E80023012044E8A7
:1093900000630E60002B1CBF0020F0E770BC70471C
:1093A00030B4044654E8000F88422CBF451A0546E5
:1093B00044E80053002BF5D1156030BC7047000025
:1093C0000648804706480047FEE7FEE7FEE7FEE75F
:1093D000FEE7FEE7FEE7FEE7FEE7FEE71D98010079
:1093E000019201002DE9F05F0546002092469B4660
:1093F00088460646814640241BE0284641464746AB
:10940000224600F067F853465A46C01A914110D3DD
:1094100011461846224600F016F82D1A67EB01088F
:109420004F4622460120002100F00DF817EB0009FD
:109430004E41201EA4F10104DFDC484631462A4695
:109440004346BDE8F09F202A04DB203A00FA02F1EF
:10945000002070479140C2F1200320FA03F3194322
:109460009040704700487047FCEC010040EA01035F
:109470009B0703D009E008C9121F08C0042AFAD2CA
:1094800003E011F8013B00F8013B521EF9D270478E
:10949000D2B201E000F8012B491EFBD27047002236
:1094A000F6E710B513460A4604461946FFF7F0FFE3
:1094B000204610BD421C10F8011B0029FBD1801A68
:1094C0007047034611F8012B00F8012B002AF9D14F
:1094D00018467047202A04DB203A21FA02F00021C6
:1094E000704721FA02F3D040C2F1200291400843B4
:1094F00019467047064C074D06E0E06840F001034E
:1095000094E8070098471034AC42F6D3FFF77CFE8E
:10951000C4F30100E4F3010070B58C1810F8015B8E
:1095200015F0070301D110F8013B2A1106D110F8FC
:10953000012B03E010F8016B01F8016B5B1EF9D100
:109540002B0705D40023521E0DD401F8013BFAE786
:1095500010F8013BCB1A921C03E013F8015B01F8F1
:10956000015B521EF9D5A142D8D3002070BD000086
:109570002DE9F04700268AB0DFF85091B0464FF44D
:109580008075012437460696284603F075F938B1F0
:10959000D9F80403204203D0284603F063F9264398
:1095A0002D1D64007F1CADB2082FEDD34FF4BE74A7
:1095B000204603F061F948B1204603F053F946F024
:1095C000004606AA0121002003F038F9404D16F0AC
:1095D000FF0F15D00127002437420DD009EB84017D
:1095E000D1F81005D1F81015C0F3042055F8242047
:1095F000C1F3014102B190477F00641C082CEBD3FA
:10960000002E5FDA4FF0FF30CDF8108054E02819BB
:1096100010F8507F90F9000027F0C008401C3BD0A4
:1096200007A9404602F080FD10B34FEA9719404663
:1096300001F0A0FE55F820701FB1B9F1030F03D05F
:1096400006E0B9F1030F27D104A9404602F074FDEA
:109650004FF0A04101EB8800D0F8000706A9C0F345
:10966000014A404602F060FD18B1BAF1020F03D082
:1096700012E0BAF1030F0FD1B9F1030F08D1BAF11B
:10968000020F1DD00221404603F0BBF8761CF6B253
:1096900017B149464046B847641C042CB7D3002E86
:1096A00010D06A460121002003F0C8F806990098FE
:1096B000884207D006900498002634460790A6E713
:1096C0000321E0E70AB0BDE8F08700000060004039
:1096D0008C2B002000F01F020121914040098000E6
:1096E00000F1E020C0F88012704700F01F02012155
:1096F00091404009800000F1E020C0F8001170475F
:1097000000F01F02012191404009800000F1E0209B
:10971000C0F8001270474907090E002806DA00F069
:109720000F0000F1E02080F8141D704700F1E020E8
:1097300080F800147047000070B54FF48076304612
:1097400002F010FE114CB50560B1304602F011FE7A
:109750000120C5F80803607920B9012060712168F3
:10976000002088474FF48276304602F0FBFD002847
:109770000AD0304602F0FDFD0220C5F8080321683A
:10978000BDE870400120084770BD00005C25002046
:1097900007480021C0F84011C0F84411C0F8481132
:1097A000C0F84C11C0F80011C0F8041104F0E6BD77
:1097B0000010014000F0B0B970B50E46144900EB3E
:1097C000400001EBC0051446E86A183520B10128B5
:1097D0000FD0022805D113E0284600F0D1F9A042AD
:1097E00001D2002411E022463146284600F000FA5A
:1097F0000BE0284600F0C4F9A042F4D20446F2E798
:109800003146284600F0C7F90446204670BD0000E6
:109810003433002004F000BD03F09ABDF0B5A84831
:10982000A74B012600781B1D1A1D4FF080510628FA
:109830000BD11C78240708D11478C4F30314032C2B
:1098400006D0042C04D0052C02D0062807D011E045
:10985000B1F824439B4DC4F304242C6002E01C782F
:10986000240707D11478C4F30314032C02D1974DB5
:10987000954C6C67D1F83051D1F84442944FC4F301
:1098800042343C6006280CD11C78240709D1147896
:10989000C4F30314032C04D18E4C276827F080777F
:1098A00027604FF080470024C7F80C41C7F81041EB
:1098B000874F3F1F3C60062807D11F783F0704D120
:1098C0001778C7F30317032F02D0062808D01FE02C
:1098D000DFF8FCC103270CF1640CCCF8007007E042
:1098E0001F783F0714D11778C7F30317032F0FD141
:1098F000DFF8E4C10527CCF80070774F78373E6079
:10990000754F08373C600CF1040C3F27CCF8007011
:10991000724F3F68DFF8C8C1CCF800706F4F3F1D31
:109920003F680CF1040CCCF800706C4F08373F68AE
:109930000CF1040CCCF80070684F0C373F680CF148
:10994000040CCCF80070654F10373F680CF1040C24
:10995000CCF80070614F14373F680CF1040CCCF860
:1099600000705E4F18373F68DFF874C10CF1200CAF
:10997000CCF80070594F1C373F680CF1040CCCF840
:109980000070564F20373F680CF1040CCCF8007083
:10999000524F24373F680CF1040CCCF800704F4F45
:1099A00028373F680CF1040CCCF800704B4F2C3773
:1099B0003F680CF1040CCCF80070484F30373F681A
:1099C000DFF81CC10CF1400CCCF80070434F343769
:1099D0003F680CF1040CCCF80070404F38373F68FA
:1099E0000CF1040CCCF800703C4F3C373F680CF194
:1099F000040CCCF80070394F40373F680CF1040C70
:109A0000CCF80070DFF8DCC0FB27CCF8007006282B
:109A100013D11F783F0710D11778C7F30317032F0F
:109A200003D0042F01D0052F07D1D1F85872DFF8E9
:109A3000B8C007F04F07CCF800702C480268D20776
:109A400002D06FF001020260062D08D1D1F8340176
:109A5000062804D12648016841F4806101604FF076
:109A60001021D1F80002002803DBD1F804020028FD
:109A700022DA204A166020480368002BFCD0152308
:109A8000C1F800320568002DFCD0C1F8043201682D
:109A90000029FCD0146001680029FCD0BFF34F8F6F
:109AA0000C48F0380168154A01F4E0611143016087
:109AB000BFF34F8F00BFFDE7124911480860F0BDAA
:109AC000E00F00F0403501400DF0ADBA00C0074096
:109AD0003C050040FCED00E010560040040400107E
:109AE00020C5004018F50040E40E0040000400408E
:109AF0003C17004004E5014000E401400400FA0581
:109B00000090D0033C2600200149024804F07EBDAD
:109B1000E82B00200020004010B5124C02202061EC
:109B2000606111A0A06104F17800E0614FF4007061
:109B300020620020A06260620BA1A164E06204F5D3
:109B40001E71E1641021A065C4E91410E06509A14B
:109B5000E01DFFF7B6FC08A12046FFF7B2FC20206D
:109B6000A07110BD343300205465726D696E616C54
:109B7000000000005254540053454747455200002E
:109B80000269C1688A4203D88068401A104400E024
:109B9000501A401E70472DE9F047C46817468946A1
:109BA00006464FF000083069A04201D9051B02E0CB
:109BB000B168201A0D1AB0686D1E001BA84200D8AB
:109BC0000546BD4200D33D4670682A4620444946BA
:109BD000FFF74CFCB0687F1B2C44A844A944A0426A
:109BE00000D10024F460002FDDD14046BDE8F087AD
:109BF0002DE9F04104468846D4E90207C51BE16817
:109C0000606816460844B54206D94146FFF72EFC67
:109C1000B819E060BDE8F0812A464146FFF726FC0E
:109C2000761B08EB050132466068FFF71FFCE66013
:109C3000F0E70000014A024900F031B817B701000F
:109C4000D425002002E008C8121F08C1002AFAD15A
:109C500070477047002001E001C1121F002AFBD1AC
:109C6000704700000121202803DA814005480140A7
:109C700003E0402802DA2038814009B10120704712
:109C800000207047FC06FFBD082806D228B1012835
:109C900003D0042801D001207047002070472DE92F
:109CA000F04116460F460446002503E03946B0470A
:109CB000641C6D1C20780028F8D12846BDE8F0818E
:109CC00010B501220221002001F064F908B1072833
:109CD00010D107220221012001F05CF908B1072808
:109CE00008D100210A22084601F054F908B10728DA
:109CF00000D1002010BD022001F056B870B500243C
:109D0000064D06E06868012110F8340003F0FAFB04
:109D1000641C28788442F5D3002070BD682500209B
:109D2000F8B515460C460646052A01D20720F8BDAF
:109D300003F0E4FC18B903F0A9FC0028F7D112499C
:109D400000224E600C708D60C1E90422C1E9062238
:109D50000E4D0DE006EBC4002968009181788DF866
:109D6000011000780A4A694603F01EFC0028DED183
:109D7000641EE4B2EED2BDE8F84004480021054A72
:109D8000001D00F07BB800006825002010EA0100EB
:109D9000A9B7010089B5010072B602F0F5FF00BF56
:109DA00002F034FE0028FBD1104C0121208801EB89
:109DB00000400FA102F03AFF10480068C00700D031
:109DC00000BE2088022101EB00400DA102F02EFF11
:109DD000BFF34F8F0948E43801680D4A01F4E06190
:109DE00011430160BFF34F8F00BFFDE76C260020D9
:109DF000466174616C206572726F7200F0ED00E074
:109E000053797374656D207265736574000000008A
:109E10000400FA050EB500210091CDE901106A4653
:109E200044F20100FFF7B8FF0EBD10B58268C368A9
:109E3000934203D001F048FC002010BD052010BD66
:109E400029B112B1531E134203D0092070470E20CE
:109E500070470160838000218160C16008467047BF
:109E600010B58268C3689A1A83889A4203D801F0B1
:109E700035FC002010BD042010BD0000074B9B786E
:109E800023B12AB120B10068037C1BB108207047C0
:109E90000720704741744261002070472C2C00203D
:109EA00070B503F0A9FF104800240B210470447022
:109EB0000E4D817014206C602C706C70FFF70AFCE2
:109EC00007211420FFF727FC1420FFF70EFC084899
:109ED000046007211120FFF71EFC0548001F0068E1
:109EE000A860002070BD00002C2C002088250020D8
:109EF000081501402DE9FC47DFF8789099F8023009
:109F000073B368B3052902D20720BDE8FC87436913
:109F100033B3437C012B25D0002704460025884617
:109F200016468DF80050684600F0C4F801A804F009
:109F300099FCC8B1012101700F4944600968C0E96A
:109F40000218C0E904769DF8040089F801009DF824
:109F5000000000F0D3F81420FFF7D2FB2846D4E726
:109F60000820D2E70F46D8E704259DF8000000F04E
:109F7000C5F8F3E72C2C0020041501400649897828
:109F800039B130B1416921B100210174022104F0DD
:109F9000D1B90820704700002C2C002070B50A4E63
:109FA00001460A48B578FFF740FF04464DB100204E
:109FB000B070711C0122C81D02F038FA08B1FFF719
:109FC00029FF204670BD00009C250020382D002070
:109FD000F0B5244E89B01F460D00044672603FD094
:109FE000A888296882B22048FFF72AFF002835D1C7
:109FF000A889A96882B21C481030FFF721FF002809
:10A000002CD1202219496846FFF730FA6069069082
:10A01000207C00B101208DF814008DF81C70607C4C
:10A0200000B10E208DF81500E0680290A068039042
:10A0300020680190606800900A480D4A694608301F
:10A0400002F0D4F9002809D1B0702068401C05D076
:10A0500004490122491CC81D02F0E8F909B0F0BD0D
:10A060000720FBE79C250020382D002020EA010076
:10A070003DE5010010B501460C48FFF7F1FE040074
:10A0800011D10B4803F04EFC68B9094907480C3957
:10A09000FFF7CBFE38B9064901220C3901F108005F
:10A0A00002F0C7F90446204610BD0000482D0020EC
:10A0B000A825002030B5EFF3108172B60D4A9468E0
:10A0C000012324B10370002900D162B630BD936032
:10A0D0004FF0E023D3F88051074C25401560C3F8BA
:10A0E0008041D3F8844154605A17C3F88421002278
:10A0F0000270E8E7582D0020FC06FFBD0B498A6876
:10A10000002A11D000280FD1EFF3108072B60B682F
:10A110004FF0E022C2F800314B68C2F8043100224F
:10A120008A60002800D162B670470000582D0020D8
:10A130002DE9F041064608680C46411C4FF0A04747
:10A140004FF0010506D005FA00F1C7F808152068A0
:10A1500002F04DFB6068411C02D0002102F03EFB82
:10A160003168A069C1F82405607D217D326808430B
:10A17000C2F86C05D4E900123068C0F80C15C0F8BC
:10A180001425207D012815D1A068411C02D0002192
:10A1900002F024FBE068411C05D08540C7F8085553
:10A1A000E06802F024FBD4E902123068C0F8082508
:10A1B000C0F81015BDE8F08170B51500044609D04F
:10A1C0000020286034B1206820B1A079800703D036
:10A1D000072070BD0E2070BD084600F025FBC0B200
:10A1E000142804D02179814203D8042070BD0520B1
:10A1F00070BDE288216800FB02102860002070BD5D
:10A200002DE9FC47002517880646158090F82D009B
:10A210001446894630B13A462146484600F018FBBC
:10A22000051E09D1B0784FF00C0A18B32088C84633
:10A23000001DB84202D95046BDE8FC87684679DF68
:10A240000028F9D12088032108F80010208819215E
:10A25000401C80B2208008F800102088401C80B28A
:10A26000208000EB0801BDF8000004F049FA2188C5
:10A2700008442080F0780222C8B1218896F9033082
:10A2800001F1030C4846BC45D5D8425421884FF013
:10A29000010C491C89B2218000F801C02188491CA9
:10A2A00089B2218009F801302088401C2080706824
:10A2B000B8B1218890F9003001F1030C4846BC4543
:10A2C000B9D8425421880A22491C89B221804254BB
:10A2D0002188491C89B2218009F801302088401C5E
:10A2E0002080308950B1CDE900474B46062202213B
:10A2F00006F1080004F0CEFA051E9DD1308A50B157
:10A30000CDE900474B460722032106F1100004F077
:10A31000C1FA051E90D1308B50B1CDE900474B46B4
:10A320001522142106F1180004F0B4FA051E83D199
:10A33000306A30B13B462246494601F0BAF8051E64
:10A34000DBD1706A30B13B462246494601F068FDD8
:10A35000051ED2D196F82C0038B13B46224649461C
:10A36000304603F06BFE051EC7D1307838B13B464E
:10A3700022464946304601F0D9FD051EBDD128468A
:10A380005AE718B504460020ADF8000013466A46A7
:10A39000204600F006F8002802D0BDF80000204456
:10A3A00018BD70B588B182B10024158803E0065D40
:10A3B000641C3444A4B2A54203D8061976789E42A0
:10A3C00001D08C42F3D38C4201D3002070BDA11C7C
:10A3D0001180005D401E80B270BD80F83010704763
:10A3E0002DE9F0410D00044606D02CB195F87A0015
:10A3F0000026012803D006E00E20BDE8F08195F884
:10A400009800012829D0D5F8A000042825D0D5F837
:10A410009C00042821D04FF00108A6702C2205F1E1
:10A420007801201DFFF722F884F83060D5F8A400E9
:10A430006063D5F8A800A0634FF6FF70A4F8A800E9
:10A4400004F19400C4F8A400C4F8AA60A4F8AE60B3
:10A4500084F8B060207810B104E00720CDE7FF2039
:10A4600084F8540004F155011F27C4F89410A4F88F
:10A47000987004F198022846FFF7C2FE0028BCD16C
:10A4800015F13C0F0ED004F17401C4F89C10A4F82F
:10A49000A07004F1A00205F13C00FFF7B1FE002816
:10A4A000ABD103E0C4F89C60A4F8A06084F85180AC
:10A4B000208BA4F8480084F83C80266484F850601F
:10A4C00060696064454604F13C02002104F15400D7
:10A4D00072DF002891D125708FE710B50288102A0D
:10A4E0001BD0112A20D0262A1DD1007A0C46012823
:10A4F00001D0022817D1A0780521401CB0FBF1F251
:10A5000001FB1201204600F052F800280BD0A16B8D
:10A51000002908D0BDE810400847C27B012A02D1BB
:10A520008088A1F8A80010BD0C46002184F8B21064
:10A530008088B4F8A8108842F5D120790028F2D19B
:10A540000121DFE710B50C46022801D0032810D105
:10A55000607800280DD000206070A178204600F0BF
:10A5600026F8002805D0A16B002902D0BDE81040D4
:10A57000084710BD10B5044690F8540074DF012060
:10A5800084F8B200002084F8B40084F8500006215A
:10A59000204601F0ACF8002808D1A178204600F050
:10A5A00006F810B1A16B01B18847002010BD2DE95C
:10A5B000F05F044600780F4638B1A770002002F023
:10A5C00041F8012620B16670F4E00820BDE8F09F54
:10A5D0000025C4F8AA50A4F8AE5084F8B050A07971
:10A5E00010B1A078012806D0E07968B1A0780128E0
:10A5F00001D0022808D1616B21B184F8B160082034
:10A60000884701E084F8B15004F1AB0100200A5CF6
:10A610000AB1304603E0401C0628F8D300204FF072
:10A6200002084FF0030A4FF0040B012F06D0022F4F
:10A630000CD0032F0FD0042F15D110E0A17929B130
:10A6400094F8241011B908B130460DE0E17911B148
:10A6500008B1404608E0207A08B1504604E0607A2C
:10A6600008B1584600E02846A070616B41B103284C
:10A6700001D0042804D1607910B194F8B200A0B1DF
:10A6800084F8B35004F13C0018210746FEF707FF99
:10A6900004F12C0084F83C60814603F0C7FA58B1FD
:10A6A00094F82C0084F8510008E084F8B45084F841
:10A6B000B36007208847E5E784F8516094F82400E8
:10A6C00050B1484603F0B2FA20B194F8280084F85B
:10A6D000520001E084F8526084F85050A27804F1EE
:10A6E000AA0104F19409052A4DD2DFE802F06503BE
:10A6F0000F1B320084F83160C4F8A450C4E910156F
:10A7000084F83C808020A4F848003EE084F8318042
:10A7100087F800A0228ABA81C4F8A4507960E16861
:10A72000B96032E06069B860208BB8813D4684F83A
:10A730003C60204604F078F840B185F8148004218C
:10A74000204600F0D4FFF0B9052115E084F831A0CF
:10A7500017E0E069B860208CB8813D4684F83C6021
:10A76000204604F061F850B185F814800421204699
:10A7700000F0BDFF38B9062184F8311001E084F8FB
:10A7800031B0C4F8A490A07878B13A4604F15400EE
:10A79000D4F8A41072DF00287FF418AF94F83010BA
:10A7A00094F8540073DF0028F6D1616B11B194F86E
:10A7B00031008847002009E784F83150F5E70000B0
:10A7C00070B5040012D001461C221448FEF74EFE5C
:10A7D0001248134D0560206850B17ADF002806D179
:10A7E0002068016829604068686005E00E2070BD3F
:10A7F0000B487BDF0028FAD108484FF6FF71143868
:10A80000084A20F8041B0549343901600021FFF78C
:10A8100035FB0028EBD0032070BD0000E42A0020A7
:10A820004C250020C1E7010010B5044600F006F8F1
:10A8300008B1204610BD142010BD0000142801D31B
:10A84000002070470146014801F0DFBB042B0020C7
:10A850007CB5054608880C460930904201D90C2089
:10A860007CBD68466DDF0028FAD121880820685435
:10A8700020881B21401C80B2208029542088401C45
:10A8800080B220802844DDF801100160BDF8051079
:10A8900081802088801D80B220809DF800104908AA
:10A8A00000D0012129542088401C208000207CBD3C
:10A8B000F8B5294D028804466E88212A37D011DC6C
:10A8C00026484FF00301102A008801EB004013D006
:10A8D000112A25D0132A29D100231A468521304672
:10A8E0007FDF17E03B2A32D0522A2AD0562A1DD1C8
:10A8F0008088132176DF0DE019A102F097F9072077
:10A9000000F06AFB08B1FFF785FAA1886980174853
:10A9100001F0B0FC002809D0BDE8F840FFF77ABA92
:10A9200013A102F083F94FF6FF706880F8BD002094
:10A930000090A08869468FDF0028F7D0FFF76AFAF9
:10A94000F8BD00231A4619463046B1DFE2E7808899
:10A95000132176DFDEE70000082500206C260020AA
:10A96000436F6E6E6563746564000000802900208B
:10A97000446973636F6E6E65637465640000000004
:10A9800010B51A4C0188606810290ED011292BD1FE
:10A99000401E606028D1FFF793F9002824D0216879
:10A9A000002921D0BDE810400847D0B9002101227C
:10A9B000084600F0EFFA08B107280FD1072202215C
:10A9C000012000F0E7FA08B1072807D1042202218C
:10A9D000002000F0DFFA20B1072802D0216801B181
:10A9E00088476068401C606010BD0000442500205E
:10A9F0002DE9F04701883B4E40F2F3194FF6FF7501
:10AA000010291BD011293ED0122954D0502946D1EB
:10AA1000C188F289841D914241D1618902293ED1C8
:10AA20008688304600F002FF050038D004F10C00A3
:10AA300000F076F9A8B3294630464EE0C17B8788FE
:10AA4000044601292BD1A846284600F0EFFE050058
:10AA500017D02F8000202872234843464A460168B9
:10AA6000C5F80A104068C5F80E0004F1100105F1A0
:10AA70000A0000F09FFF6872F08900280FD1294674
:10AA80002AE0042013E0808800F0D0FE040006D005
:10AA90006068FFF773FA08B103F0A0FA2580BDE8FB
:10AAA000F087FFE76868FFF769FA0028F7D0BDE88C
:10AAB000F04703F093BA87880646384600F0B6FEA2
:10AAC0000400ECD02B464A4606F1080104F10A00C6
:10AAD00000F070FF607221463846BDE8F04700F094
:10AAE0002FBD0000E42A00204C2500202DE9F04F66
:10AAF0000746858802883D48012197B08346102A81
:10AB000009D0112A49D01A2A6CD1387AB1EB101F1A
:10AB100045D2012244E0354C083CA068C0430B906C
:10AB200061680BA801F092FA0B990CA800F0A2FC46
:10AB30002C220CA96846FEF799FC0026E946A0469F
:10AB400010E000BF09EB46005FF00004B0F804A07D
:10AB500008EB84005146001D01F04CFA641C1D2CCA
:10AB6000F6D3761C0098B042ECD8142D05D317B05C
:10AB70000420BDE8F04FFFF74DB92946584601F0D3
:10AB80004FFA294608F1040001F04AFAF87B01283F
:10AB900028D016482946001D15E029461AE0002253
:10ABA0000221B1EB101F01D2012600E000260F495F
:10ABB000083901F11000041D294682B101F030FA74
:10ABC00036B12946204617B0BDE8F04F01F028BA4B
:10ABD0002946204617B0BDE8F04F01F00BBA01F04E
:10ABE00009FAF5E717B0BDE8F08F0000082B002048
:10ABF000F0B585B016460F4604001D4614D004AAD1
:10AC000019466069FFF7D8FA00280BD1A5F57F40F7
:10AC1000FF380BD0049848B1007848B13088F42848
:10AC200008D9072005B0F0BD0E20FBE70520F9E7A5
:10AC30000820F7E700200090019002900390A08880
:10AC4000ADF8000001208DF80200CDE902676946E9
:10AC50002846AEDFE6E7000030B5144B0D46040091
:10AC60000FCB85B08DE80F001ED0EDB12868A06134
:10AC70002146684662DF002814D120788DF8120042
:10AC80000120ADF81000A21C04A9A8DF002809D1FA
:10AC90002946204603F0CEF8002803D12946204655
:10ACA00003F0A6FB05B030BD0E20FBE7F8E901007C
:10ACB00070B588B00446002924D0002C22D0084664
:10ACC0002188102920D0502924D057291AD105468F
:10ACD000A188406906AAFFF76FFA002812D1069EE4
:10ACE000307800280ED018216846FEF7D8FB0120E6
:10ACF0008DF800000195A088ADF808000396A969B9
:10AD00006846884708B070BD08B02146BDE870406D
:10AD100002F07EBE08B02146BDE8704002F044BF9C
:10AD2000007800F0010070470149085C704700009E
:10AD3000B8E901000649095C4FF0A040D0F81005C1
:10AD4000C84010F0010000D0012080F001007047E1
:10AD5000B8E901002DE9FC410646C0074FF00005A7
:10AD60000ED0104F00240122385D009500231146BB
:10AD7000019501F0FDFC641C042CF4D300F046F8AE
:10AD8000B0070DD5074E0024361D0022305D032389
:10AD900000951146019501F0EBFC641C042CF4D3E2
:10ADA000BDE8FC81B4E9010007490B5C4FF0A0410C
:10ADB000D1F804250120984020EA0203C1F80835A3
:10ADC0001040C1F80C057047B4E901000249085C65
:10ADD000012101F027BD0000B4E901000249085C2F
:10ADE000002101F01FBD0000B4E901000649095C23
:10ADF0004FF0A040D0F80405C84010F0010000D08A
:10AE0000012080F001007047B4E9010010B5002472
:10AE10002046FFF7DBFF641C042CF9D310BD10B5EE
:10AE200000242046FFF7DAFF641C042CF9D310BD80
:10AE300010B50246064B4FF0FF3000215C5C944297
:10AE400001D1084610BD491C0429F7D310BD0000EC
:10AE5000B8E9010070B50C4E0C004FF000053060F1
:10AE60000BD0012000F06AF808B1022004E00020B5
:10AE700000F064F800B10B202070706810B9FEF784
:10AE80001FFF0546284670BD4425002010B5002050
:10AE900000F0D4F908B1062806D1012000F0CEF95F
:10AEA00008B1062800D1002010BD00002DE9F047B0
:10AEB0000D468146FFF7BCFF0446042836D2DFF872
:10AEC00074801B481C4EA8F10C0725B3012D0ED031
:10AED000022D2BD104EB440030444578002D25D0C1
:10AEE000B968002922D02846BDE8F047084704EB9E
:10AEF0004401755C0E44717849B10E4A4FF400412B
:10AF0000093A8068FEF7F6FF08B987F80390B17830
:10AF100008F80410E2E78068FFF730F804EB44011A
:10AF2000314418F804008D78A842D7D0BDE8F087E6
:10AF3000BCE9010040250020842A0020042801D219
:10AF4000FFF7F8BE002070470146104810B5408852
:10AF5000042907D007290ED00A2915D1BDE81040D1
:10AF600003F0B0B8132176DF0CE000280CD0BDE868
:10AF70001040FEF74FBFA0F57F41FF3904D10448D0
:10AF8000FFF7F8FA0828F0D110BD000008250020CE
:10AF90008C29002070B50023042810D20D4D00EB41
:10AFA0004004012A02D101290CD00022094E00EBF5
:10AFB0004000304461B1012906D0022906D00723A0
:10AFC000184670BD0E30C2B22A55F9E74270F7E755
:10AFD0008270F5E7842A0020044A01460020127995
:10AFE000D20702D0084600F04DB870473425002043
:10AFF00070B506461E480024C0E90161B00720D59F
:10B000000025012211462846FFF7C4FF6D1C0446A7
:10B01000042D02D2002CF4D013E094B940F2666201
:10B0200004211448FEF77CFE04000AD1FEF766FEF8
:10B03000040006D10F48104A0021001FFEF71EFF32
:10B040000446F00712D00120FFF784FE74B90948C6
:10B050000A4A00210C38FEF711FF040006D105480A
:10B06000074A01210838FEF709FF0446204670BD53
:10B0700034250020C8E9010009B3010029BA010004
:10B08000F79C01002DE9F05F6A4C054600266078C8
:10B09000B34618B184F801B000F0AEFC664F4FF42F
:10B0A0007A694FF4C87A4FF00108182D62D2DFE8B0
:10B0B00005F0AC0C0C31404D62676B746B74BE7D57
:10B0C0007D7D7D7DACAFB2B5BEBE0020FFF78EFEAC
:10B0D00000284FF0000008D0FFF778FE022D02D1C3
:10B0E0004FF4E16008E0484606E0FFF777FE022DE6
:10B0F00001D1C82000E05046410CC0034FF4FA7261
:10B10000801841F10001257052000023FEF76AF912
:10B1100001462AE00020FFF769FE00284FF00000FA
:10B1200004D0FFF753FE4FF44870E5E7FFF756FEF3
:10B13000DFE70020FFF75AFE00284FF0000002D0A2
:10B14000FFF744FECFE7FFF749FED4E70020FFF703
:10B150004DFE00284FF0000002D0FFF737FE01E05F
:10B16000FFF73CFE257041F69A1100223868FEF781
:10B17000C1FE064646E00020FFF716FE257008E0F7
:10B18000002051E025703DE084F801800120FFF7A8
:10B190000BFE002240F6CD41E8E784F80180012053
:10B1A000FFF702FE00224FF48041DFE77868FEF7E8
:10B1B000E5FE0646D5F1110000D02EB10220FFF7C2
:10B1C00005FE84F802B01DE0012816D980B2C8211E
:10B1D0004843C117C90341EA5041C0034FF4FA7212
:10B1E000801841F1000152000023FEF7FBF80146F0
:10B1F00000227868FEF77EFE06460220FFF7EEFD8D
:10B2000084F802803046BDE8F09F00F0F5FBB9E716
:10B2100000F0F2FBB4E700F0EFFB04E000F0ECFB21
:10B220000020FFF7DBFD0120FFF7D8FDAAE7FFF7BD
:10B23000F6FDA7E734250020BCE90100012103F059
:10B2400090BB00002DE9F8430546861C00208DF8D0
:10B25000000090460F464FF001096846FEF72AFFAE
:10B260001B4C20683860D4E90001401AA16804F240
:10B270001C47081A0EE00121384600F0E1FE00F0FC
:10B2800061FC0146384600F0DBFED4E90001401ABB
:10B29000A168081A401C8642EDD8B8F1000F03D00F
:10B2A000052065F3891002E0062065F39F50A2682F
:10B2B0002168114004EB8101C8602068304420609F
:10B2C0009DF80000FEF71AFF4846BDE8F88300002D
:10B2D000102F002030B482680468531C8360A1548E
:10B2E000D0E901128A4202D330BC01F0B2B830BCBE
:10B2F00070470000034803C8814201D10120704714
:10B3000000207047102F002000780221FFF7CEBDEB
:10B3100005494FF0FF32082841F8202002D30844A5
:10B3200080F84820704700008C2B0020F0B54FF0CB
:10B33000FF3512B10023082601E008230C260C4C2F
:10B3400005E000BF54F823707F1C04D05B1CB3429F
:10B35000F8D32846F0BD26185DB286F8305044F880
:10B360002310002AF5D1E11881F84800F1E7000028
:10B370008C2B00200249084490F9300070470000EF
:10B380008C2B002070B5084C050009D010342168C2
:10B39000002907D008682060496828468847F6E7F2
:10B3A0000834F4E770BD0000782B0020054A012125
:10B3B00020B1012805D19170FFF7E4BF5170002042
:10B3C000FAE77047782B00202DE9F05F26484168A6
:10B3D000F1B3DFF898B00E688146DBF8004087686B
:10B3E0008078E11B21F07F45ED1CB0B9DFF880804B
:10B3F0004FF48030C8F84403C8F804031120FEF766
:10B4000069F91120FEF771F94FF0010AC8F800A0A0
:10B410002F2002F06FF889F802A0B54200D235461D
:10B42000124BE8193C3320F07F401860DBF8001025
:10B430005A46091B21F07F41001B20F07F40C91CA8
:10B4400081420FD9106818602F2002F053F800E0F5
:10B4500004E0BDE8F05F1120FEF752B9BDE8F05FEF
:10B4600002F0CABCBDE8F09F882500200415014009
:10B470000010014073B58CB00646002000900D9876
:10B4800080B100246D4621460DA800F0BEFD30B10C
:10B49000009805EB400084800098401C0090641CDC
:10B4A000142CF0D32C2269463046FDF7DFFF0EB096
:10B4B00070BD2DE9F04117880646B81D14460D46AB
:10B4C000984202D90C20BDE8F08131880722062974
:10B4D0000AD34FF4486C4FF6FF73614501D9994286
:10B4E00002D17088062801D21046ECE7604501D9E8
:10B4F0009842F9D1994203D0984201D08142F3D8C1
:10B500000520E85520881221401C80B22080295453
:10B510002088401C80B220804119308803F0F0F868
:10B520002188084480B220804119708803F0E8F82F
:10B530002188084420800020C5E7FEF76BBC00008E
:10B5400038B54A7A0F4B62B100220A725969002954
:10B5500006D001228DF80020ADF802006846884729
:10B5600038BD0A7A62B19B684C680246194620468B
:10B57000FEF7C0FC0028F3D0BDE8384002F02EBD35
:10B580005B68F1E7E42A00202DE9F0470025DFF8A9
:10B590008C803CE06068002100EBC5060120327819
:10B5A0009146FDF750FFD4E9062300EA020701EABD
:10B5B000030C57EA0C0728D082438B434846C4E962
:10B5C000062302F059F83278824691460120002184
:10B5D000FDF739FFD4E9042300EA020401EA030776
:10B5E0004A4650460021FDF72EFF44404F403C4361
:10B5F0000BD17078012801D0012100E00021726890
:10B6000081EA0A010AB1484690476D1CEDB298F8EC
:10B61000000044468542BDD3BDE8F0876825002080
:10B6200010B50021024800F01CFD80F3100010BD91
:10B630002C3300200E4910B50A784C780023A24222
:10B6400012D0521CD2B20A70022A00D10B70084AE2
:10B650000B780C3252F8232002608868104420F0E6
:10B660007F408860012010BD0360002010BD0000F5
:10B670008825002030B50446006887B00D468068F4
:10B6800000281FD018216846FDF709FF0195A06822
:10B690000590207910B1012810D107E001208DF824
:10B6A000000020690290E068039005E002208DF818
:10B6B0000000E068000302906069049020688168DF
:10B6C0006846884707B030BD826883881A4003689F
:10B6D0009A5C0A708168491C81607047C2688388DF
:10B6E0001A4003689954C168491CC160704770B51D
:10B6F0000D460446B0F89810D0F894000122FEF7E9
:10B7000040FE00B1057004F13C0204F1940104F123
:10B71000540072DF70BD10B50446C0B2FEF7AAFC3B
:10B72000204610BD0B484A8843889A4211D10A88A6
:10B73000A2F52063773B0CD18988C91E8AB282802A
:10B74000054803211346008801EB004003A101F0E6
:10B7500078BA7047082500206C2600204461746187
:10B76000206C656E2069732073657420746F2030BF
:10B77000782558282564290010B50949094800F0A2
:10B78000F1FC08B1FEF746FBF721064800F0DEFCAD
:10B79000002803D0BDE81040FEF73CBB10BD000000
:10B7A00025B70100702900202DE9F04180460246AE
:10B7B00001200021FDF747FE1A4F05460E46786826
:10B7C000FEF7DCFB00280CD1174CD4E9062110460B
:10B7D0002A4001EA06031A4305D0A843B143C4E94D
:10B7E0000601BDE8F081404601F046FF30B1D4E9E2
:10B7F000040128433143C4E9040105E0D4E90410FD
:10B80000A943B043C4E90410D4E9060128433143F5
:10B81000C4E90601A1687868BDE8F0410022FEF79E
:10B8200069BB000010EA01006825002001460348BA
:10B8300002888A4200D0002070470000D02A0020F1
:10B840002DE9FC5F0E008346DDE90C47C6F10000E0
:10B8500098469246814600D40846012503E000BF81
:10B8600090FBFAF06D1C5045FADAA84500D9454620
:10B8700024B1002E01DB780700D5641EB80702D57D
:10B88000B8F1000F0AD0F80708D13CB1A54205D2A3
:10B8900020215846641EFFF71DFDF6E7002E02DA50
:10B8A0004E462D2102E0780703D52B215846FFF79D
:10B8B00011FD07F0030002280BD1B8F1000F08D1E9
:10B8C0003CB1A54205D230215846641EFFF702FD67
:10B8D000F6E7CDE90047434652463146584602F066
:10B8E00015FFBDE8FC9F000070B50D4604460068DA
:10B8F0004FF4887101F0C3FD4FF49071206801F09E
:10B90000BEFD4FF49271206801F0B9FD4FF4A271B1
:10B91000206801F0B4FD20681249C0F804132068C3
:10B920006907000B40B2090E002806DA00F00F008C
:10B9300000F1E02080F8141D03E000F1E02080F821
:10B94000001420680121000B40B200F01F0291405A
:10B950004009800000F1E020C0F88012C0F800111A
:10B9600070BD000010030200024600201268930719
:10B9700002D0530702D47047500714D502F00300D9
:10B98000012802D002280CD105E0C2F383100B6815
:10B99000801C184404E00223086803EB9252104410
:10B9A000086001207047086800EB9253C2F38910C9
:10B9B000401CEEE7F0B58488A518944200D82246D2
:10B9C000A41AC288D6189A4200D81346D21A4B88B5
:10B9D0000788BB420CD34088834209D88888A0429C
:10B9E00006D3A84204D8C888904201D3B04201D9F6
:10B9F0000020F0BD0120F0BD0A4810B5807860B18C
:10BA0000002401E0022C06D02046FFF7DFF9641C79
:10BA1000042CF7D310BD0324F6E7BDE81040FFF770
:10BA2000F5B900003425002003480179C90702D088
:10BA30000078FFF727BB704734250020F7210180ED
:10BA40001721418000210171417170472DE9F047B4
:10BA5000394E002780463D46DFF8E090D6F804A036
:10BA600057E003D00446D0F81C8035E099F8002058
:10BA700002EB4201521CD2B289F8002009EBC1014D
:10BA800099F80230091D9A4201D189F8005048689E
:10BA90000A780446012A12D0022A02D0032A3BD196
:10BAA00008E002F017FC00B10127257434E00574AA
:10BAB000C06900E070680028F9D170602CE0207C3B
:10BAC00050BB88686060C868A0600869E060486929
:10BAD000A061F07800B165606268B168184B501AD7
:10BAE00020F07F40984202D2A168084406E0881AFC
:10BAF000A16820F07F40814202D9081A206000E04E
:10BB0000256065600120A56020742046E56102F093
:10BB1000C3FBB8F10000A4D199F8001099F8010016
:10BB20008142A3D117B97168514502D00120BDE807
:10BB3000F0870020FBE70000882500202C2C002047
:10BB4000FFFF7F002DE9FF410026234800F075FA32
:10BB50002148001F074600F070FA204C60680090F2
:10BB6000A56800E000986946284004EB80000C308E
:10BB7000FFF7FAFE0028F5D101AA009901EA0503B2
:10BB800004EB8303491CDB6842F82030401C009121
:10BB90000228F2D3019800F0030001280BD00228FC
:10BBA00010D10198032101EB90500099BDF80A6073
:10BBB00001EB900005E00198BDF80A60C0F3831026
:10BBC00008440090384600F035FA08B100986060EB
:10BBD00004B03046BDE8F08128330020102F00204B
:10BBE000ACB018226E496846FDF740FC6D480690DF
:10BBF0006D494FF48070CDE90701099007236B4A26
:10BC000006A96846FEF7E4F908B1FEF703F94FF418
:10BC10000041002001F074F808B1FEF7FBF800F0D5
:10BC2000E7FEFEF73DF908B1FEF7F4F8604903209E
:10BC3000FFF7DEF908B1FEF7EDF869460020FFF7DF
:10BC400009F908B1FEF7E6F801F078F908B1FEF756
:10BC5000E1F801F035FB08B1FEF7DCF80024694695
:10BC60000120009401F094F908B1FEF7D3F868467A
:10BC700001F036FA08B1FEF7CDF89DF808004DA1A5
:10BC800020F00F00401C20F0F00010308DF808006C
:10BC90000B2202A87CDF08B1FEF7BCF8009410204C
:10BCA000ADF800003C200194ADF80200ADF804406E
:10BCB0004FF4C870ADF8060068467ADF08B1FEF7A9
:10BCC000A9F8FFF759FD3E48019001A93D4800F051
:10BCD000DCFA08B1FEF79EF83B48009069463B4805
:10BCE000FEF7BAFF08B1FEF795F8AC216846FDF7FC
:10BCF000D6FB02208DF800008DF8024005208DF85B
:10BD000003000120ADF84C0030498DF87C00402044
:10BD1000891F2290149144F2506023902C4829905E
:10BD2000284869460C30FEF75BFB08B1FEF772F855
:10BD3000244801210C30FEF750FB1C216846FDF71A
:10BD4000AEFB4FF42030CDE900404FF4702002905C
:10BD500020480590032520488DF80C500690ADF83A
:10BD60000E408DF810406846FEF72AFD08B1FEF738
:10BD700051F81AA0FDF75EFF1D481EA1008805EBD3
:10BD8000004000F053FF0F4803210C30FEF70FFC7A
:10BD900008B1FEF73FF800F039FE01F0E3F8FAE7EA
:10BDA0009CE901007027002070280020CDE40100EC
:10BDB00049AF01004E6F726469635F554152540090
:10BDC00079CF01008029002041D9010014250020ED
:10BDD000D1D90100F5D901003BB501000D0A55414B
:10BDE000525420737461727465642E0D0A00000051
:10BDF0006C2600204465627567206C6F6767696E0A
:10BE00006720666F722055415254206F766572200C
:10BE100052545420737461727465642E00000000E3
:10BE200070B5144682880E4605462088111D0144CF
:10BE3000921C994201D8FE2A01D90C2070BD521CD7
:10BE400032542088FF21401C80B220803154208849
:10BE5000401C80B220808119288802F051FC218882
:10BE6000084480B22080AA8842B1A96841B1304418
:10BE7000FDF7FCFA2088A98808442080002070BDC6
:10BE8000072070BD2DE9F047C7880446181D1646E7
:10BE90008946B0FBF7F1B0FBF7F207FB12009A19E5
:10BEA0003A44D21CB2FBF7F2DDF820A001E024688E
:10BEB000491E0029FBD13D1A8846B54216D818E024
:10BEC000BAF1000F05D0211809EB08002A46091D18
:10BED00004E0204409EB08012A46001DFDF7C6FADC
:10BEE00000202468761BA844B74201D9354600E0FB
:10BEF0003D46002EE4D1BDE8F087000030B5024693
:10BF000059B100F029FF0021074C09E004EB81033F
:10BF100015685B88AB4202D11160002030BD491C1E
:10BF20008142F3D3052030BD40260020F8B50F46EE
:10BF3000017814460546012901D1687830B120887E
:10BF4000821C9A422DD8012902D006E00720F8BDB4
:10BF500069780144891C994223D8181A801E86B238
:10BF6000ADF800602188B81C084469467DDF0028D0
:10BF7000EDD12878022805D1BDF80010B14201D8D2
:10BF800009210AE00821012805D16878B04202D8C9
:10BF9000ADF8000001E0ADF80060BDF80000FE283B
:10BFA00001D90C20F8BD2288401CB8542088401CC0
:10BFB00080B2208039542088401C2080BDF80010B9
:10BFC000084420800020F8BD10B50A8849888A42BC
:10BFD00003D1FDF761F9012010BD002010BD70B53F
:10BFE0000C460546FDF73BF9002802D06188286819
:10BFF000084470BD01F01F0301229A40D243490951
:10C0000000EB8100114600F021B84A0950F82200E7
:10C0100001F01F0201219140084000D0012070472B
:10C0200001F01F0301229A40490900EB81001146EB
:10C0300000F01CB8002100F00FB8012100F016B884
:10C0400008B56A46FDF77DF9009808BD08B56A464F
:10C05000FDF75DF9009808BD08B56A46FDF757F988
:10C0600008BD08B56A46FDF739F908BD08B56A4646
:10C07000FDF740F9009808BD08B56A46FDF76EF96E
:10C08000009808BD38B5044600258DF80050684674
:10C09000FEF710F821686268086890420ED9401EC9
:10C0A00008600178A38AE26801FB0325227A2168EF
:10C0B000101AC0B20A79824200D208719DF80000BD
:10C0C000FEF71CF8284638BD38B5054600208DF827
:10C0D00000000C466846FDF7EDFFE868A98A201AC3
:10C0E000B0FBF1F12A681068431C136001709DF8E1
:10C0F0000000FEF703F838BD10B530B1017A426890
:10C100000368891AC9B21A6006E00E2010BD0368E0
:10C110001A68541C1C601170491EC9B2F7D200681D
:10C1200000210171084610BDC20800F0070301207C
:10C13000895C98400840704710B5C20800F00703BA
:10C14000885C01249C402043885410BD28B1A1F193
:10C150001702E12A03D3072070470E2070470180A1
:10C160000020704710B560B1C160F72120F8021BB4
:10C1700020F8021BFB2100F8021BFFF75FFC0020E8
:10C1800010BD0E2010BD00007CB50C468188002932
:10C1900033D102880025102A06D0112A09D03A2A64
:10C1A0000BD0552A2ED129E00146204601F066FC2D
:10C1B00028E0A01DFFF742FC24E02246408934F825
:10C1C000063F834200D818466080172800D2172007
:10C1D0006080D06878B1607968B1174BD3E900030B
:10C1E000CDE90003ADF802106088ADF80400D36813
:10C1F000694610469847657125717CBD0146204609
:10C2000001F07EFCA07A0028F7D02846E188A5DF5F
:10C21000012670B11128F0D001F022F9024607483A
:10C2200007A1008802B006EB0040BDE8704000F0B6
:10C2300001BDA572E6727CBDE8E901004026002040
:10C2400073645F626C655F67617474635F65786374
:10C2500068616E67655F6D74755F72657175657332
:10C260007428292072657475726E65642025732E9A
:10C270000000000020B10278DE2A03D008207047B9
:10C280000E20704741800020704760B159B102789C
:10C29000DE2A0AD009684160DE2101704FF6FF7185
:10C2A0004180002070470E207047082070477FB5FE
:10C2B000054600294DD0002D4BD008780C46DE28CD
:10C2C00047D1A8886188884202D1204602F0B8FA96
:10C2D0002888012825D002283BD011283AD051289F
:10C2E00037D135F8040F6188884232D1A978A81C6B
:10C2F00002292ED1017A042903D0062901D005296B
:10C3000027D10021009102228DF8002001914FF4E5
:10C31000C07202910391ADF80420007A05280FD075
:10C3200010E0297A2046012913D1A9884288914238
:10C330000FD10121017204B0BDE8704002F080BA53
:10C34000ADF8041028886946B0DF002801D0616884
:10C3500088477FBDA88861888842FAD14FF6FF7070
:10C3600060807FBD00F180400068002800D001207F
:10C37000704708B500F1804000210160006800901E
:10C3800008BD000070B50B4C207808B185250FE082
:10C390000020A06060602061E060074801F08CF838
:10C3A000054600F0E7FF08B901F070F801202070A1
:10C3B000284670BD782B0020ADB3010038B50025AC
:10C3C0008DF800506846FDF775FE074CE068401E8A
:10C3D000E060E06810B901F07FF8A5709DF80000FA
:10C3E000FDF78CFE38BD0000782B002070B50646A6
:10C3F00004780C4888B0154640F82420094A08699A
:10C40000121D42F8240020226846FDF72FF80494FC
:10C410000DB1054A00E000226946301D01F082F9A5
:10C4200008B070BD54250020DDE50100001D01F0BD
:10C43000AFB9001D01F02EBA0FB408B50399002959
:10C4400004D004AA00926A4600F00FF801B05DF82B
:10C4500014FB10B582680446002A05D0D4E9040311
:10C46000216898470020A06010BD2DE9FC47914647
:10C470000C00804676D014F8011B39B125290ED066
:10C480004046FEF727FF20780028F4D198F80C00EA
:10C49000002867D04046BDE8FC47FFF7DABF002020
:10C4A000012221782B291BD02D2902D0302908D137
:10C4B00002E040F0010001E040F00200641C002AAC
:10C4C000EFD100252A290ED02178A1F130020A2AC5
:10C4D00011D205EB850201EB4205641C303DF1E70A
:10C4E00040F00400EAE7D9F800100B1DC9F800304D
:10C4F0000968641C0D44217800232E290BD114F8FF
:10C50000011FA1F130020A2A05D203EB830201EBDD
:10C510004203303BF3E76C290DD068290BD0692921
:10C5200021D00BDC252918D0582931D063290ED011
:10C53000642915D117E014F8011FECE7702969D0C0
:10C54000732932D075291BD0782909D120E0D9F878
:10C550000000011DC9F8001001784046FEF7BAFE40
:10C56000641C90E76CE0D9F800100A1DC9F800209F
:10C570000968CDE900500A224046FFF761F9EFE76C
:10C58000D9F800100A1DC9F8002009680A2206E03F
:10C59000D9F800100A1DC9F8002009681022CDE959
:10C5A0000050404602F0B2F8DAE7D9F80010002750
:10C5B0000A1DC9F800200E68C00705D112E04046E8
:10C5C000761C7F1CFEF786FE31780029F7D104E047
:10C5D000202140466D1EFEF77DFEBD42C0D9002DD4
:10C5E000F6D1BDE74EB13046FCF764FF074604E0E4
:10C5F000202140466D1EFEF76DFEBD4206D9002D7E
:10C60000F6D103E04046761CFEF764FE317800293F
:10C61000F8D1A5E7D9F80000011DC9F80010056898
:10C6200030214046FEF756FE78214046FEF752FE86
:10C6300008200021CDE90001034610222946B0E779
:10C64000BDE8FC872DE9F04128B1016819B1C9693D
:10C65000BDE8F04108470D4D0D480024461B142746
:10C660000DE000BF04EB840005EB8000016829B1F8
:10C67000C969884710B10120BDE8F081641CB6FB90
:10C68000F7F0A042EED80020F6E70000000000001E
:10C6900000000000044801214174007A08B1002024
:10C6A0007047012070470000F02D0020012801D0C4
:10C6B000032808D10449002201284A7400D0002030
:10C6C000087401F049BB7047F02D002070B5024698
:10C6D000022801D0032A45D1234C207A002841D0DA
:10C6E000012833D0022831D120480023022A0068D3
:10C6F00002D0032A2AD11BE0E360017911B101299C
:10C7000024D10DE0D0E90565711B4FF48056B1428C
:10C7100000D33146294481614569A9420ED015E014
:10C720000169491C0161426991420FD1237213E0F2
:10C73000E168491CE160082908D9E3602372022AF4
:10C740000AD00D21FEF796FF01F0FCFA607C28B1BB
:10C75000BDE8704000F014BE0021F3E7BDE8704072
:10C7600001F0FABA70BD0000F02D0020C4250020B1
:10C7700070B541EA4201DDE904564FF0A04441EAB8
:10C78000830141EA052104EB800041EA0641C0F83B
:10C79000001770BD70B541EA4201DDE904564FF063
:10C7A000A04441EA830141EA052104EB800041EA0B
:10C7B0000641C0F8001770BD70B541EA4201DDE9DD
:10C7C00004564FF0A04441EA830141EA052104EBFD
:10C7D000800041EA0641C0F8001770BD1CB5002278
:10C7E0000B46009211460192FFF7E6FF1CBD1CB5F7
:10C7F000002100910B46012201911146FFF7DCFF59
:10C800001CBD4FF0A04202EB8000D0F8002722F4BC
:10C810004032C0F80027D0F8002742EA0141C0F8B2
:10C820000017704701224FF0A043824011B1C3F8B6
:10C8300008257047C3F80C257047000018B5084B51
:10C840006C4601441B68009306E000BF54F820309A
:10C85000D3F81035401C08C28142F7D818BD00003B
:10C8600008EA0100034908B5084400210160006896
:10C87000009008BD0060004002494058012800D0E7
:10C88000002070470060004030B5124B0146002088
:10C89000D3F81044224609E0157A854205D1401CA0
:10C8A0000A28F7DB4FF0FF3030BD5268002AF3D181
:10C8B000421CF9D00872D3F810242AB152684A6099
:10C8C000D3F81024516030BD0022C3F810144A6020
:10C8D00030BD0000102F00207047FCF76BBF704781
:10C8E00008B5034A00924023024A00F005F808BD4B
:10C8F000EDDF0100102E0020F0B595B01C46154666
:10C900000F4608461A9E00F0F7FA182109A8FCF70E
:10C91000C6FD0E96CDE909540023082203A9384626
:10C9200000F0FFFA05980690BDF81000ADF81C0065
:10C93000BDF81200ADF81E0000208DF8210003980C
:10C94000082600F00300012802D0022818D032E0A7
:10C9500003983346850AC0F3C2008DF8200003987F
:10C960000FA9C0F38314A200384600F0DAFA09A830
:10C97000009006AB22460FA9284600F019FA1AE0EB
:10C980000398840DC0F3C2008DF82000082C01D25A
:10C99000254600E0082533462A460FA9384600F010
:10C9A000C0FA2E44641B09AB06AA29460FA800F062
:10C9B00051F9002CEAD1384600F0A4FA15B0F0BDC8
:10C9C0000A4A012902EBC00007D0022907D0032937
:10C9D00007D0042907D000207047022070470420A8
:10C9E000704700797047407970470000E4F3010018
:10C9F00010B5FFF772FF04210348FFF745FF024916
:10CA00000120487210BD0000DC2500202DE9F04F08
:10CA10008DB0FEF76FFC18B100200DB0BDE8F08FAF
:10CA20007A4C4FF0000BC4F818B4BFF34F8F606816
:10CA30000290A568D846284004EB800008E02168F1
:10CA40000298814201D86160E6E7284004EB80004B
:10CA50000C3002A9FEF788FF0028F0D105AA029940
:10CA600001EA050304EB8303491CDB6842F820302C
:10CA7000401C02910228F2D3059800F0030002281E
:10CA800002D001284ED0A9E005985022810D894698
:10CA9000B2EB905F00D850210E4666F39F50059090
:10CAA00008315B4800F0DFF9070079D000F024FA84
:10CAB0004346082205A9384600F039FA029908F1E0
:10CAC000080A2940681A8000001D864223D94F4D6C
:10CAD0000C3530B1C2B204EB8101301A90460C31F2
:10CAE00004E02946F2B2002590462846C6B25346D5
:10CAF000384600F01CFA0AEB08032DB132462946ED
:10CB00004FEA070000F013FA029909F1030001EB64
:10CB1000900002903BE004EB8101534632463846D8
:10CB20000C31EFE70598C0F38310062800D30620E8
:10CB3000059960F38911C1F38310801C0591810070
:10CB4000334800F090F9070048D000F0D5F943468B
:10CB5000082205A9384600F0EAF908F1080800267D
:10CB60000FE00298434600EA0501401C04EB8101F6
:10CB70000290042238460C3100F0D9F908F104087B
:10CB8000761C0598C0F38310B042EAD847B1D4F8B8
:10CB90001054D4F8180468B1384600F0B3F92FE007
:10CBA0001CE0687A012804D12A68284639461268B0
:10CBB00090476D68002DF4D1384600F0A3F98DF848
:10CBC00000B06846FDF776FAD4F8180408B9029860
:10CBD00060609DF80000FDF791FA11E0D4F8104470
:10CBE00004E021682046896888476468002CF8D1F1
:10CBF00008480221008801EB004007A100F016F868
:10CC0000FEF778FB80F0010007E70000102F0020FE
:10CC10005CF401006C2600204261636B656E6473F6
:10CC200020666C75736865640000000000231A4676
:10CC300001F0ACBA08B5012300926A4601F0A6FAE9
:10CC400008BD1CB5CDE9002302236A4601F09EFA17
:10CC50001CBD00002DE9F0470E4680461C4692465A
:10CC600008293ED894F80C900020207319461046ED
:10CC700001F01CF80025B54206D218F805201AA1CB
:10CC80002046FFF7D9FB03E019A12046FFF7D4FBAC
:10CC90006D1C082DEFD317A12046FFF7CDFB002513
:10CCA000B54210D218F80570FCF7DCFB0068C05DD7
:10CCB00010F03E0F01D03A4600E02E220EA1204691
:10CCC000FFF7BAFB03E00DA12046FFF7B5FB6D1C93
:10CCD000082DE5D301222146504600F0C9FF84F813
:10CCE0000C90BDE8F087000020253032780000006D
:10CCF000202020007C0000002563000020000000B0
:10CD0000104810B5FF218160002101604160C0F82A
:10CD10001814C0F8141480F820140B4800F0F0F830
:10CD200000280DD109480A490A4B401AC1080020C1
:10CD300003E000BF23F82000401C8842FAD3002003
:10CD400010BD0000102F00205CF401005CF4010015
:10CD5000E4F301004026002002480349401AC008BD
:10CD6000704700005CF40100E4F3010013B568466D
:10CD7000FFF7C4F808B100201CBD0248009950F824
:10CD800031001CBDE4F3010070B508480125D0F85E
:10CD9000104480F8205405E06572216820464968F7
:10CDA00088476468002CF7D170BD0000102F002068
:10CDB0002DE9FF4781460C9D00200C462F7B2873F0
:10CDC000984616462946184600F070FF072E42D2B4
:10CDD000DFE806F004090F161F2A360049462846E8
:10CDE000FFF72AFB37E0494628462268FFF724FB75
:10CDF00031E0D4E9002349462846FFF71DFB2AE02D
:10CE0000A0680090D4E9002349462846FFF714FBA8
:10CE100021E0D4E90201CDE90001D4E9002349462B
:10CE20002846FFF709FB16E004F1080007C88DE863
:10CE30000700D4E9002349462846FFF7FDFA0AE037
:10CE400004F108000FC88DE80F00D4E9002349461B
:10CE50002846FFF7F1FA00222946404600F008FF75
:10CE60002F73BDE8FF872DE9F041858A80462D1F8D
:10CE70004819C01CB0FBF5F0C6B24046FFF702F9F6
:10CE8000041E19D00020207101206071E580002768
:10CE90002546761EC4F800800BE04046FFF7F2F806
:10CEA00060B16179491C6171286005467F1CC0F83A
:10CEB0000080B742F1D32046BDE8F081204600F063
:10CEC00002F80020F8E72DE9F041457901466B1E94
:10CED000002201E00968521C9A42FBD30F68014608
:10CEE000002605E038460C68FFF7EEF82146761C70
:10CEF000AE42F7D3BDE8F0810121001DFFF7A0B8D5
:10CF0000FFF7FAB810B504460121001DFFF7B4F889
:10CF100010F0FF0F04D12046BDE81040FFF7D3BF4B
:10CF200010BD38B501240094FEF7ACFF38BD38B50C
:10CF300000240094FEF7A6FF38BD0000064910B596
:10CF400000204870091D0860BFF35F8F0349044843
:10CF500000F042FA002010BDCC25002078EA010044
:10CF6000042E002010B500F005FA08B141DF10BD15
:10CF700020BF40BF20BF10BDFCF74CBF20B103490C
:10CF800009680160002070470E2070474CEC0100DA
:10CF90002DE9FE4306460D460846FFF7EFFF002841
:10CFA0007ED18046CDF80080CDF804800124062093
:10CFB0008DF80060ADF80400CDF808808DF80240CF
:10CFC000694620202A6869DF3E4F40B100F048FAE8
:10CFD000024638883C4904EB0040FFF72BFECDF8B1
:10CFE0000080CDF80480CDF808808DF801406946B6
:10CFF00040202A6869DF40B100F032FA02463888E2
:10D00000324904EB0040FFF715FECDF800808DF8A3
:10D010000060F720ADF80200CDF80480CDF808805C
:10D02000694623202A6869DF40B100F019FA0246F8
:10D030003888274904EB0040FFF7FCFDCDF800805D
:10D04000CDF80480CDF808808DF80040464669464A
:10D0500001202A6869DF40B100F002FA02463888F0
:10D060001C4904EB0040FFF7E5FD4FF4B060009071
:10D07000019602966946A1202A6869DF48B100F04E
:10D08000EFF93988024604EB014313491846FFF7CC
:10D09000D1FD0096019602968DF80060694600E089
:10D0A0000DE0A0202A6869DF40B100F0D9F90246FE
:10D0B00038880A4904EB0040FFF7BCFD0020BDE8BA
:10D0C000FE8300007426002048F2010090F2010067
:10D0D000DCF20100A8F10100F4F1010054F10100BB
:10D0E0002DE9F0410446D0F8008060DF2168194D39
:10D0F000074641451CD92888022606EB004016A1A8
:10D10000FFF794FD2888424606EB00401EA12368E5
:10D11000FFF797FDF006D0F80C012168800200F1BE
:10D120000050421A288825A106EB0040FFF782FD37
:10D13000012467B1384600F093F9024628882AA1F5
:10D1400004EB0040FFF776FD3846BDE8F0812E483D
:10D150000470F9E774260020496E7375666669638A
:10D1600069656E742052414D20616C6C6F6361740F
:10D17000656420666F722074686520536F6674441E
:10D1800065766963652E00004368616E676520748B
:10D1900068652052414D207374617274206C6F6316
:10D1A0006174696F6E2066726F6D2030782578200B
:10D1B000746F20307825782E000000004D6178696A
:10D1C0006D756D2052414D2073697A6520666F72CE
:10D1D000206170706C69636174696F6E206973207F
:10D1E000307825782E00000073645F626C655F659F
:10D1F0006E61626C6528292072657475726E656453
:10D200002025732E000000003B26002030B5154875
:10D21000ADF5017D0078002821D04FF4FA7500BFEC
:10D22000ADF8005280A9684661DF38B1052816D0F4
:10D230000DF5017DBDE83040FCF7ECBD6C460A49B8
:10D240007DA800F0C9F806E0D0E90021204690470B
:10D250007DA800F0D8F87F980028E1D0F4E70DF51C
:10D26000017D30BD3B26002050EC0100F8B5134C89
:10D270002078C0B10120A07000F082FE112814D0E7
:10D28000022000F095FE00258DF800506846FCF75E
:10D2900011FF11DF064625709DF80000FCF72EFFF8
:10D2A0002EB13046F8BD0820F8BD0020F8BDA570AD
:10D2B00000F028FF032000F07BFEF6E73826002070
:10D2C0007CB5204C207808B108207CBD0120A070DE
:10D2D000002000F055FE112819D0002000F068FE53
:10D2E00019480026006801908DF800606846FCF738
:10D2F000E1FE164901A810DF05000AD000202070C9
:10D300009DF80000FCF7FAFE2DB128467CBD0020F8
:10D310007CBD0120F3E7A67066700721162000F09F
:10D32000E6FD08B1FCF776FD0721152000F0DFFDD2
:10D3300008B1FCF76FFD00F001FF012000F038FE9E
:10D34000E5E7000038260020E4EB0100999D01008C
:10D350000EB50749684600F03FF805E0D0E9001037
:10D360008847684600F04FF802980028F6D10EBDB5
:10D3700000EC0100014800787047000038260020CA
:10D380000548817819B1007818B1FFF76FBF082000
:10D390007047FFF795BF0000382600201FB568468C
:10D3A0004BDF30B1052814D004B0BDE81040FCF7C5
:10D3B00031BD084901A800F00FF806E0D0E90021CE
:10D3C0000098904701A800F01EF803980028E6D0C6
:10D3D000F4E71FBD6CEC0100016009684160AFF328
:10D3E000008010B5D0E900215368994201D1002195
:10D3F00004E0D1E90034A34202D01946816010BD97
:10D4000008314160F0E7816800290BD0026892681A
:10D410000A44826041684B689A4203D108314160F6
:10D42000FFF7DFBF704700000C4A10B502F5947398
:10D430000EE0991AC91001EBD171491002EBC1013C
:10D440000C68844201D90B4602E005D201F10802C2
:10D450009A42EED3002010BD486810BD98EA010042
:10D4600000B5FFF7E1FF002800D1014800BD000032
:10D4700084EA01004058002800D00120704708B518
:10D48000002242504058009008BD00000848006843
:10D49000012110F0010F08D14FF0E020E02280F8C8
:10D4A0000024C0F88012C0F80011024801607047E3
:10D4B00000E100E0180500400649024600200B7913
:10D4C0000BB1852070470A6001220A7100224A715F
:10D4D000704700005C2500200449012008600448D2
:10D4E0000168C1F300410029FAD170470C000040E7
:10D4F00018040040002802D0014980010847704705
:10D5000019EA01002DE9F0418846054600F098FB34
:10D51000234E002828461AD0FDF72CFF304490F8FF
:10D5200048008009032802D001280ED007E04FF000
:10D53000A040D0F81005E84010F0010F05D00321FD
:10D540002846BDE8F041FFF75CB90221F8E700F09A
:10D5500083FB002822D02846FDF70CFF04464FF439
:10D56000807000EB84000F4F81B207EB8400D0F88D
:10D57000102542F00102C0F810250846FFF772F9A5
:10D58000B8F1000F0AD02846FDF7F4FE56F8200047
:10D59000002803D00120A040C7F80403BDE8F081B3
:10D5A0008C2B0020006000402DE9FC41DFF8BC809E
:10D5B000044608EB0400002790F930001346C0171A
:10D5C0000E46401C01D008274CE0B0781946C0F345
:10D5D00040022046FDF7AAFE0546401C41D0B07827
:10D5E000410719D4C0070AD04FF0A04000EB8401D6
:10D5F000D1F8000720F00200C1F8000707E0002181
:10D600007378204600910A460191FFF7C3F8174945
:10D6100020465431FEF790FDB078800718D51448A5
:10D62000317800EB8500D0F81025124B1A40C0F875
:10D6300010254FF4F8524FF4403302EA042203EA73
:10D6400001410A43D0F810150A43C0F8102509E03B
:10D6500008EB0500327810F8481F41EA821101708A
:10D6600000E004273846BDE8FC8100008C2B002038
:10D6700000600040FFE0FCFF4FF0A041D1F8101522
:10D68000C14011F0010000D00120704770B5184D65
:10D6900095F8580008B1082070BD0020411E2A18D6
:10D6A000401CC0B282F830102028F8D30024204655
:10D6B000FDF72EFE641CE4B20C2CF8D300240D49B7
:10D6C000E0206C6581F8000401264020891FC1F824
:10D6D0008002C1F800014FF4BE70FFF7C3F806499D
:10D6E000F007C1F8040385F85860204670BD0000BB
:10D6F0008C2B002006E000E000600040034890F81A
:10D700005800002800D00120704700008C2B00201A
:10D710000121B1EB507F01D10120704700207047FB
:10D72000002070472DE9F0410546164600790F4666
:10D73000154A00EBC00102EB810494F8201011B1EE
:10D740000820BDE8F081114951F820102868FFF742
:10D75000E7FF08B11120F4E739462846FCF7E8FC5A
:10D760006660386920601EB1397F2846FEF7BCF834
:10D7700028680821C0F800150020A061E06101219F
:10D78000606184F82010DCE7E82B00200CEA01003F
:10D790002DE9F05F044600790E4600EBC001DFF88A
:10D7A000F0A017460AEB81053046FFF7B1FFB0B194
:10D7B00068684FF000084FF4047910B12168C1F88F
:10D7C0000893A8694FF0000B80B1E86948B1686818
:10D7D00010B12068C0F804931120BDE8F09F10201C
:10D7E000FBE7EF614FF001082E6102E0EE60C5E952
:10D7F000067B00254FF488712068FFF740FE4FF448
:10D80000A2712068FFF73BFE2068C0F83465C0F8BD
:10D8100038752068B8F1000F12D0D0F8001241F02E
:10D820002001C0F800122079D04600EBC0010AEBBD
:10D830008100406838B12068C0F804932846CCE7DE
:10D8400001210160EFE74FF4887A4FF4A279514645
:10D850002068FFF70FFE074649462068FFF70AFEDB
:10D8600006464FF492712068FFF704FE014647EA2E
:10D8700006000843EBD0227902EBC20308EB8302D7
:10D88000C2F818B001B10325002ED7D00F25D5E777
:10D89000E82B00202DE9F04704460E460079204988
:10D8A00000EBC00001EB800517463046FFF730FF64
:10D8B00030B1204600F036F820B11120BDE8F087E5
:10D8C0001020FBE76F61AE604FF490760027314681
:10D8D0002068FFF7D4FD4FF4AC7841462068FFF78D
:10D8E000CEFD2068AA686969C0F84425C0F84815CB
:10D8F000206801218160686878B9B146494620688E
:10D90000FFF7B8FD064641462068FFF7B3FD064322
:10D91000F4D000B10F27002068613846CEE7000040
:10D92000E82B00200079054900EBC00001EB8000E6
:10D930004069002800D0012070470000E82B00203B
:10D940002DE9F04105460078002826D10026144F25
:10D950004FF0010812E02869805DFCF78BFB0400A2
:10D960000BD0112CF7D03988224608EB01400DA1CD
:10D97000FFF760F92046FCF74DFA761CA88AB04202
:10D98000E9D8A98A2869084410F8010C0D2804D1A7
:10D990000A20FCF76FFB1128FAD0BDE8F0810000E7
:10D9A0006C2600204661696C656420726563656958
:10D9B00076696E67204E5553206D65737361676598
:10D9C0002E204572726F7220307825782E2000004C
:10D9D00010B550B103280CD10220FDF7FDFA002844
:10D9E00007D0BDE81040FCF715BABDE8104000F0C4
:10D9F00069BB10BD0078002807D104483B2140884E
:10DA000076DF002801D0FCF705BA70470825002012
:10DA1000F0B58BB0002601960D4604468988406912
:10DA200001AAFCF7C9FB0AA8CDE908600227ADF8F6
:10DA30002070ADF82260218AA88808AAADDF0028EE
:10DA400019D1A069002816D00998FDF769F90028B6
:10DA500011D0019E0EB101203070182102A8FBF7F1
:10DA60001EFD8DF808700394A888ADF81000059687
:10DA7000A16902A888470BB0F0BD000070B502464E
:10DA80008888C97B00EB400302EB4304A41D0129F5
:10DA900001D11188218021886288914211D9A5DFA6
:10DAA000012568B111280DD0FFF7DAFC02460648BF
:10DAB00006A1008805EB0040BDE87040FFF7BAB84A
:10DAC000657170BD257170BD4026002073645F6272
:10DAD0006C655F67617474635F65786368616E67C6
:10DAE000655F6D74755F7265717565737428292043
:10DAF00072657475726E65642025732E00000000D7
:10DB00007CB506468D88C88805EB450106EB4104C7
:10DB1000A41D172800D217202188814200D808466A
:10DB200060800020207121882846B5DF50B1FFF7C2
:10DB300097FC02460E480121008801EB00400DA130
:10DB4000FFF778F86079002810D1F06800280DD030
:10DB50001449D1E90201CDE90001ADF80250608815
:10DB6000ADF80400F2686946304690477CBD00007D
:10DB70004026002073645F626C655F676174747334
:10DB80005F65786368616E67655F6D74755F726508
:10DB9000706C7928292072657475726E6564202511
:10DBA000732E0000E8E90100F0B587B00C46054689
:10DBB0008E1D8988406906AAFCF7FEFA182168467E
:10DBC000FBF76DFC0195A088069AADF8080003925A
:10DBD00031882B89002704F11200994202D1738900
:10DBE000022B0DD0AA8991421ED1A96900291BD010
:10DBF0008DF8007004907089ADF81400A96911E0E7
:10DC0000002A11D0FDF78CF820B106990120087088
:10DC1000022002E00698077003208DF80000A96931
:10DC2000002901D06846884707B0F0BD0068012888
:10DC300003D0022801D00020704701207047000067
:10DC40000449084490F93000082801DB012070479E
:10DC5000002070478C2B00200449084490F93000C4
:10DC6000082801D201207047002070478C2B00202B
:10DC700010B50C46017A052908D0407A38B1084819
:10DC800008A102682046FEF7D7FB00E01AB106A102
:10DC90002046FEF7D1FB2046BDE81040FEF7D9BB79
:10DCA00014260020257300000D0A000038B5C38833
:10DCB0000D46044633B114A0009015A216A12846C3
:10DCC000FEF7BAFB217A05291CD0607A48B1A088FA
:10DCD000FEF776FE164951F8202016A12846FEF7D9
:10DCE000ABFBA0880021FFF741F803461049207ADA
:10DCF000143951F8202001B02846BDE830400EA16B
:10DD0000FEF79ABB38BD00001B5B306D00000000C1
:10DD10001B5B313B33316D0025734C6F677320649F
:10DD2000726F70706564202825642925730D0A00C0
:10DD300014260020257300003C25733E2025733AED
:10DD400020000000034802490068FEF73DB90000CA
:10DD5000C825002050EA01002DE9F041234C0025A0
:10DD6000234E207A012730B92248311D0068FEF782
:10DD700036F9306038B1022020723168087928B154
:10DD800001281ED116E06560BDE8F081D1E90503E8
:10DD9000C01A4FF48052904200D31046B7EB900F58
:10DDA00001D2820800E001220869C96818441944B8
:10DDB00029DF03E0D1E90301084428DF58B1112825
:10DDC00012D003213068FDF755FC25726560BDE86F
:10DDD000F041FFF7B7BF207C0028D5D1BDE8F04166
:10DDE00000210220FEF772BC2772CDE7F02D002043
:10DDF000C425002050EA010070B5012670044FF0E0
:10DE0000E0210025C1F88001084C4010C4F8480307
:10DE1000C4F8080366602F20FFF76CFBA660044C73
:10DE20002F20A560FFF766FBA57070BD00100140B4
:10DE30008825002030B58FB005461C216846FBF7C9
:10DE40002EFB00249DF80000019440F00C008DF89A
:10DE50000000039404940594069428788DF8360005
:10DE60000220ADF834000C949DF83000142120F00D
:10DE70000F00401C20F0F00010308DF830009DF8AD
:10DE8000310020F00F00401C20F0F00010308DF821
:10DE900031009DF8320020F00600801C20F01800B0
:10DEA00040F001008DF8320007A8FBF7F8FA0DA842
:10DEB00007900CA808900120ADF82400F420ADF8DC
:10DEC0002640ADF82800688805F10C0307AA6946CA
:10DED000AADF0FB030BD1FB501238DF800308DF8DB
:10DEE00008100192D0E90012684690471FBD70B536
:10DEF0000D460446FBF7B6FE70B12846FBF7C4FE9C
:10DF000068B16807000E002C0CDA04F00F0101F173
:10DF1000E02181F8140D09E042F2010070BD42F2E7
:10DF2000020070BD04F1E02484F80004002070BDFC
:10DF300038B50021012548B101280CD0032809D1AA
:10DF4000FFF7A4FABDE83840FEF738BA4FF0E020FA
:10DF5000C0F8805138BD8DF800106846FCF7AAF86B
:10DF6000064C207808B9FEF70DFAE068401CE06026
:10DF7000A5709DF80000FCF7C1F838BD782B002093
:10DF80003EB5044609496846FFF726FA08E000BF97
:10DF9000D0E900212046904730B16846FFF733FAB8
:10DFA00002980028F4D13EBD11203EBDE8EB0100EF
:10DFB0003EB5044608496846FFF70EFA07E000BF81
:10DFC000D0E90021204690476846FFF71CFA0298E6
:10DFD0000028F5D13EBD0000F4EB0100024989693B
:10DFE000002900D008477047E42A00202DE9F041BD
:10DFF0001400884618D000250E4F032608EB0501B3
:10E0000022460020FBF7D8FB0544241A40B9387893
:10E01000002809D008494FF47A408847761E05D079
:10E0200001203870002CE9D1BDE8F0810020387063
:10E03000FAE70000D8250020CDEB01002DE9F041E2
:10E040000746806A14468846C8B3002531E000BF01
:10E05000B96A05EB450001EB8006B088801CFE28FC
:10E0600002D90C20BDE8F0812288401C08F802008B
:10E0700020881622401C80B2208008F800202088CA
:10E08000401C80B2208000EB0801308800F038FB93
:10E090002188084480B22080B28842B1B16871B151
:10E0A0004044FBF7E3F92088B188084420806D1CC8
:10E0B000EDB297F82C00A842CAD80020D2E7FFE7BB
:10E0C0000720CFE710B50020FCF786FF08B1FBF76B
:10E0D000A1FEFCF7DBFE08B1FBF79CFE33DF002856
:10E0E00003D0BDE81040FBF795BE10BD002805D158
:10E0F0000349012048700020FDF744B97047000033
:10E10000782B002010B51620FBF7ACFD48B10A486B
:10E1100082684FF4800152B1016821F480010160EE
:10E1200010BDBDE8104042F20100FBF773BE4FF096
:10E13000E020C0F8801110BD582D002010B5162029
:10E14000FBF790FD80B10F4890F800044009FBF701
:10E150009BFD60B10C4882684FF480016AB1016890
:10E1600041F48001016010BD42F2010001E042F281
:10E170000200BDE81040FBF74DBE4FF0E020C0F8B4
:10E18000001110BD16E000E0582D00202DE9F84FD9
:10E19000204D924689460646984601226946184611
:10E1A000AF68FDF74FF858B3009800210446801C73
:10E1B00009E000BF00EA07035AF8212005EB8303BA
:10E1C000401C491CDA604145F4D34FEA164AFDF77A
:10E1D00027FA4AEA0041601C384005EB80003C40C9
:10E1E00005EB8402C160D06866F3C50068F389104E
:10E1F00069F39F2020F00300401C20F00400D06051
:10E2000095F8200402E000BFFEF700FC0028FBD1D7
:10E21000BDE8F88F102F00202DE9F84F1D4C002588
:10E220006846D4E901A6FDF705FA002738B30023B4
:10E23000009A61681CE0D1F800C00846944503D9F3
:10E24000ACEB02020A6015E0A2EB0C02634407602B
:10E25000D0F80CC0C1698146BCF1000F08D006EBB4
:10E26000030828F07F48C0E9018CC9F81C50054616
:10E270000029E0D128466160FDF7E8FB03E028466D
:10E28000FDF7E4FB10B15046FDF79EF8E770BDE8DE
:10E29000F88F0000882500200D4B10B5596831B16A
:10E2A00002680C68A24204D8A21A0A60C1615860D0
:10E2B00010BD0B4603E00B46C969121B21B10C6867
:10E2C0009442F8D3A41A0C600260C161D86110BDF9
:10E2D000882500202DE9F041144E77683D462C46F4
:10E2E00003E0844204D02546E469002CF9D11BE008
:10E2F000D4B1A5420BD1F869706040B90C49012036
:10E3000088600021B160F0702F20FFF7F3F82168DA
:10E31000E069E86110B102681144016070688742E9
:10E3200002D00120BDE8F0810020FBE78825002015
:10E33000001001407CB5064600240D468DF80040D3
:10E340006846FBF7B7FE01A800F08CFA70B10570C3
:10E35000094946609DF8040048709DF80000FBF7ED
:10E36000CDFE1420FBF7CCF920467CBD04249DF89B
:10E370000000FBF7C3FEF7E72C2C00202DE9F0414D
:10E38000194D6C68002C2CD0184800270068A9682B
:10E39000B846401A20F07F462068B0420CD821468B
:10E3A000361A0744E469087C20B181F81080886936
:10E3B00049698847002CEFD129786878814206D1D5
:10E3C000401CC0B26870022801D185F8018006485F
:10E3D00069780C3040F82170BDE8F0411420FBF75B
:10E3E0008FB9BDE8F08100008825002004150140A8
:10E3F00030B58FB00024054607949DF81C001C2101
:10E4000020F00F00401C20F0F00010308DF81C00B0
:10E410009DF81D0020F00F00401C20F0F00010308F
:10E420008DF81D009DF81E0020F00600801C8DF860
:10E430001E006846FBF733F89DF80000019440F099
:10E4400010008DF8000007A8CDE90440039406945D
:10E4500028788DF83A000320ADF838000D949DF827
:10E460003400142120F00F00401C20F0F000103088
:10E470008DF834009DF8350020F00F00401C20F08E
:10E48000F00010308DF835009DF8360020F00600C1
:10E49000801C20F0180040F001008DF8360008A81C
:10E4A000FAF7FDFF0EA808900DA809900120ADF81D
:10E4B0002800F420ADF82A40ADF82C0068882B1D08
:10E4C00008AA6946AADF0FB030BD000038B5017850
:10E4D00041B1012901D002292BD14068BDE8384063
:10E4E000FBF798BC144C134D20782844FBF756FDDD
:10E4F0002078401CC0B22918207011F8011C0A298C
:10E5000002D0A188884214D32078ADF800000A48D0
:10E5100063886A4607490C30FCF76AFB082806D076
:10E520001128F1D0052802D008B1FBF773FC0020B8
:10E53000207038BD7C260020082500207CB501789D
:10E54000244D81B301290BD002292BD18DF8001065
:10E55000C068691C01900122C81DFDF767FF2EE00D
:10E56000406801781C48FBF77BFC1B4C012618B166
:10E570008DF80060019006E0A068E168814205D056
:10E5800000208DF80000696868468847A068E16847
:10E59000081AA188884207D80E490122491CC81DC3
:10E5A000FDF744FF7CBD01E0AE70FBE70A48094976
:10E5B0001030FBF73AFC30B103208DF80000696899
:10E5C00068468847EEE70349012201F10800FDF79C
:10E5D00030FFE7E79C250020382D00201FB50A46B4
:10E5E00001788DF8001041680191017A8DF80810CA
:10E5F000C0680390044850F82210001F50F82220F1
:10E60000684690471FBD0000582500202DE9FF41B6
:10E610000C464FF4927705463946FEF72BFF00264D
:10E62000C0B139462846FEF72AFF02208DF80000C7
:10E63000D5F88004C5F880040390D5F83C058DF822
:10E640000800E0680190A661E661D4E9001268461E
:10E65000904723E04FF4887739462846FEF70AFFB3
:10E66000E0B139462846FEF70AFFD5F83C15A06907
:10E67000884213D1E06960B1E268D5F8000220F069
:10E680002000C5F80002E069A0612069E661E06051
:10E6900001E0A661E2682046FFF71DFC4FF4A27777
:10E6A00039462846FEF7E6FE60B139462846FEF7B1
:10E6B000E6FEA06930B1A661D5F83C152046E268B7
:10E6C000FFF709FC4FF4907739462846FEF7D2FE53
:10E6D000002813D039462846FEF7D1FE606900288D
:10E6E0000CD0D5F84C058DF800608DF80800A068B6
:10E6F00001906661D4E9001268469047BDE8FF8149
:10E700000870000A48700220704700002DE9F05F91
:10E710008346DDE90A4A994690460D460846012798
:10E7200003E000BFB0FBF8F07F1C4045FAD2B945CA
:10E7300000D94F465FEACA7012D18CB15FEA8A7085
:10E7400002D5B9F1000F01D0202607E0302605E000
:10E7500031465846641EFCF7BDFD0CB1A742F7D305
:10E760005FF00106B9F1010F02D9A9F1010903E037
:10E77000B5FBF6F0404502D306FB08F6F2E7DFF8FA
:10E780003C9000BFB5FBF6F000FB165519F80010E1
:10E790005846FCF79FFDB6FBF8F6002EF2D15FEA73
:10E7A000CA7009D0002C07D0A74205D220215846B4
:10E7B000641EFCF78FFDF5E7BDE8F09F40EA01001D
:10E7C000F8B5054680B2FDF731F8040013D0154EB8
:10E7D000207A0027317B88420ED2A8B204F10A01C8
:10E7E00075DF28B1112806D0BDE8F840FFF7F6BB69
:10E7F000207A401C2072F8BD2772307C38B1A8B254
:10E800003B2176DF18B1082801D0FFF7E7FB7169DB
:10E810000029F0D08DF80070ADF8025068468847A6
:10E82000F8BD0000E42A0020417939B190F8B21017
:10E8300021B990F8B40008B101207047002070475A
:10E8400030B40446007A00280AD06088002166DFD0
:10E8500028B1112802D0616830BC0847012020721D
:10E8600030BC70470A494A788B78521CD2B2934226
:10E8700000D100220B78934201D100207047027032
:10E88000487800EB400001EBC000001D704700001D
:10E890002C2C00202DE9FC411646DDE90854CDE979
:10E8A00000541F468046022200F00CF8002807D1D1
:10E8B000CDE900543B4610223146404600F002F8B4
:10E8C000BDE8FC812DE9FC5F0026DDE90C4B994693
:10E8D00092468E4680462788354630E0D8F80400B8
:10E8E000002200EB850069460068019001A864DF02
:10E8F000002830D19DF8000050451FD10EB10021F5
:10E9000000E00221228808441118594522D846B94E
:10E91000521C90B2208009F800E02088401C208022
:10E920000126218801A801EB0902694664DF00285D
:10E9300011D120889DF80010084420806D1CB8F883
:10E940000000A842CADC56B12088C01B401E80B21D
:10E95000FF2802D90C20BDE8FC9F09F80700002021
:10E96000F9E710B5042817D209B1032400E0002408
:10E97000FCF7DAF94FF0A04101EB8000D0F8001766
:10E9800021F44031C0F80017D0F8001741EA0441E3
:10E99000C0F80017002010BD062010BD08000000C0
:10E9A0000600000005000000070000000000000055
:10E9B0000000D601111213140D0E0F10442A00206E
:10E9C000642A0020902A00200D000300ADAE010053
:10E9D0000E000300ADAE01000F000300ADAE01005C
:10E9E00010000300ADAE0100770A00000000000037
:10E9F000770A0000000000009ECADC240EE5A9E0B2
:10EA000093F3A3B50000406E00000050099B010085
:10EA1000030000000C2C00200738FDD870470000D0
:10EA2000FFFFFFFFFFFFFFFFFFFFFFFFFFFFFFFFF6
:10EA300000000000000000000000D60107000000F8
:10EA40003031323334353637383941424344454624
:10EA5000B0250020001000000400000001000000AC
:10EA600000000000000000000000000000000000A6
:10EA7000000000000000000060EA010078EA0100E8
:10EA800004000000556E6B6E6F776E206572726FBA
:10EA90007220636F646500000000000078F00100E0
:10EAA0000100000024EF01000200000018ED010049
:10EAB0000300000098EF010004000000ECEF0100EB
:10EAC00005000000CCEE01000600000068EE010029
:10EAD00007000000D4EF010008000000E0EE010094
:10EAE0000900000044EF01000A00000060F001008E
:10EAF0000B00000000ED01000C000000F8EE01002A
:10EB00000D000000C8F001000E000000C4EF01007D
:10EB10000F00000000F001001000000034F00100C0
:10EB200011000000DCF0010012000000B0F0010054
:10EB3000130000004CF001008000000080EE010096
:10EB400081000000BCED0100820000007CED0100AE
:10EB5000830000005CED01008400000098ED0100DE
:10EB600085000000A4EE010086000000ACEF01006B
:10EB70009000000048EE0100910000003CED010013
:10EB8000920000000CEF01000082000014F0010070
:10EB90000182000060EF0100028200007CEF0100B2
:10EBA00000840000D8ED01000184000084F0010021
:10EBB0000284000020EE010003840000FCED01004F
:10EBC000E1C80100DFC80100D9C801000738FDD83D
:10EBD00070470000B4F40100BCF401000000000024
:10EBE0000000000001000007D4EB0100E4EB01008D
:10EBF000080000000CEC01001CEC01000800000003
:10EC00001CEC01002CEC010008000000E4F4010001
:10EC1000F4F401000000000000000000D4F4010042
:10EC2000E4F40100000000000000000074F40100A2
:10EC30007CF401007CF401009CF401009CF40100D0
:10EC4000ACF40100ACF40100B4F401000025002094
:10EC50002CEC01004CEC010008000000BCF40100A9
:10EC6000CCF40100CCF40100D4F401005CEC010010
:10EC70006CEC010008000000004040404040404073
:10EC8000404041414141414040404040404040407F
:10EC90004040404040404040400502020202020223
:10ECA0000202020202020202022020202020202072
:10ECB0002020200202020202020290909090909086
:10ECC0001010101010101010101010101010101044
:10ECD00010101010020202020202888888888888B8
:10ECE00008080808080808080808080808080808A4
:10ECF00008080808020202024000000079EC010046
:10ED00004E52465F4552524F525F494E56414C4912
:10ED1000445F4441544100004E52465F4552524FB9
:10ED2000525F534F46544445564943455F4E4F54F6
:10ED30005F454E41424C4544000000004E52465F44
:10ED40004552524F525F464541545552455F4E4FD2
:10ED5000545F454E41424C45440000004E52465FD0
:10ED60004552524F525F4D555445585F554E4C4F8A
:10ED7000434B5F4641494C45440000004E52465FBC
:10ED80004552524F525F4D555445585F4C4F434B7F
:10ED90005F4641494C4544004E52465F4552524FF2
:10EDA000525F4D555445585F434F4E445F494E495D
:10EDB000545F4641494C4544000000004E52465FB6
:10EDC0004552524F525F4D555445585F494E495434
:10EDD0005F4641494C4544004E52465F4552524FB2
:10EDE000525F424C455F495053505F52585F504B01
:10EDF000545F5452554E4341544544004E52465F71
:10EE00004552524F525F424C455F495053505F50FC
:10EE10004545525F52454A45435445440000000071
:10EE20004E52465F4552524F525F424C455F4950E9
:10EE300053505F4C494E4B5F444953434F4E4E45F0
:10EE400043544544000000004E52465F4552524F25
:10EE5000525F4150495F4E4F545F494D504C454DB4
:10EE6000454E5445440000004E52465F4552524FB5
:10EE7000525F4E4F545F535550504F5254454400CB
:10EE80004E52465F4552524F525F4D4F44554C458E
:10EE90005F4E4F545F494E495449414C495A45448D
:10EEA000000000004E52465F4552524F525F4D4F98
:10EEB00044554C455F414C52454144595F494E4988
:10EEC0005449414C495A4544000000004E52465FA7
:10EED0004552524F525F4E4F545F464F554E44007D
:10EEE0004E52465F4552524F525F494E56414C4931
:10EEF000445F5354415445004E52465F4552524F71
:10EF0000525F444154415F53495A45004E52465F57
:10EF10004552524F525F494F5F50454E44494E470C
:10EF2000000000004E52465F4552524F525F53560A
:10EF3000435F48414E444C45525F4D495353494EFF
:10EF4000470000004E52465F4552524F525F494EB5
:10EF500056414C49445F4C454E4754480000000020
:10EF60004E52465F4552524F525F4452565F54577D
:10EF7000495F4552525F414E41434B004E52465FFE
:10EF80004552524F525F4452565F5457495F455263
:10EF9000525F444E41434B004E52465F4552524FE2
:10EFA000525F494E5445524E414C00004E52465F0E
:10EFB0004552524F525F53544F524147455F465559
:10EFC0004C4C00004E52465F4552524F525F4E55D8
:10EFD0004C4C00004E52465F4552524F525F494ED4
:10EFE00056414C49445F504152414D004E52465F9C
:10EFF0004552524F525F4E4F5F4D454D000000004D
:10F000004E52465F4552524F525F464F524249441C
:10F0100044454E004E52465F4552524F525F445255
:10F02000565F5457495F4552525F4F5645525255AD
:10F030004E0000004E52465F4552524F525F494EBD
:10F0400056414C49445F4144445200004E52465F91
:10F050004552524F525F5245534F5552434553000C
:10F060004E52465F4552524F525F494E56414C49AF
:10F07000445F464C414753004E52465F535543430D
:10F08000455353004E52465F4552524F525F424CD9
:10F09000455F495053505F4348414E4E454C5F4198
:10F0A0004C52454144595F45584953545300000060
:10F0B0004E52465F4552524F525F434F4E4E5F4352
:10F0C0004F554E54000000004E52465F4552524F7D
:10F0D000525F54494D454F55540000004E52465F13
:10F0E0004552524F525F4255535900007761726E3C
:10F0F000696E670064656275670000001B5B313BE9
:10F1000033306D001B5B306D000000001B5B313B3A
:10F1100033316D001B5B313B33326D001B5B313B88
:10F1200033336D001B5B313B33346D001B5B313B74
:10F1300033356D001B5B313B33366D001B5B313B60
:10F1400033376D00696E666F000000006572726F84
:10F150007200000073645F626C655F6366675F7373
:10F16000657428292072657475726E656420257334
:10F17000207768656E20617474656D7074696E6760
:10F1800020746F2073657420424C455F474154548E
:10F19000535F4346475F534552564943455F434893
:10F1A000414E4745442E000073645F626C655F63A7
:10F1B00066675F73657428292072657475726E6561
:10F1C00064202573207768656E20617474656D70A6
:10F1D00074696E6720746F2073657420424C455FBC
:10F1E000434F4D4D4F4E5F4346475F56535F555516
:10F1F00049442E0073645F626C655F6366675F738A
:10F20000657428292072657475726E656420257393
:10F21000207768656E20617474656D7074696E67BF
:10F2200020746F2073657420424C455F47415454ED
:10F23000535F4346475F415454525F5441425F53CA
:10F24000495A452E0000000073645F626C655F637D
:10F2500066675F73657428292072657475726E65C0
:10F2600064202573207768656E20617474656D7005
:10F2700074696E6720746F2073657420424C455F1B
:10F28000434F4E4E5F4346475F4741502E000000BC
:10F2900073645F626C655F6366675F73657428297A
:10F2A0002072657475726E656420257320776865B9
:10F2B0006E20617474656D7074696E6720746F2060
:10F2C00073657420424C455F4741505F4346475F3A
:10F2D000524F4C455F434F554E542E0073645F624E
:10F2E0006C655F6366675F73657428292072657457
:10F2F00075726E6564202573207768656E20617471
:10F3000074656D7074696E6720746F207365742006
:10F31000424C455F434F4E4E5F4346475F47415423
:10F32000542E00006E72665F626C655F6761747474
:10F3300000000000626C655F6E757300636C6F6344
:10F340006B000000434C4F434B0000004750494FB7
:10F35000544500005052530055415254450000009E
:10F360006E72665F6673746F72616765000000009D
:10F3700061746669666F2E6D5F6669666F00000076
:10F380007077725F6D676D740000000062616C6C75
:10F390006F632E6C6F675F6D656D706F6F6C0000D3
:10F3A000617070006E72665F736468006E72665F93
:10F3B0007364685F626C65006E72665F7364685F39
:10F3C000736F6300F4F40100002500207C0100004D
:10F3D0001895010048F501007C2600204417000024
:10F3E000549C010024F301000000030334F30100E6
:10F3F000000000003CF301000000000044F30100A5
:10F40000000000004CF301000000000054F3010074
:10F410000000000058F301000000000060F301004C
:10F420000000030370F301000000000380F30100FB
:10F43000000000008CF3010000000003A0F30100B5
:10F4400000000303A4F3010000000303ACF3010078
:10F4500000000303B8F3010000000303F0250020BF
:10F46000E8250020F0250020502E002068260020EE
:10F4700018000000EDAA01000000000089C1010091
:10F4800070290020DBA401008C29002081A9010043
:10F4900000000000F1A9010000000000B1AC010073
:10F4A00014250020AFC2010080290020B1A801006E
:10F4B0000000000095C6010000000000EDE0010022
:10F4C00000000000CDC601000000000045A50100BD
:10F4D0008C2900200DD20100000000009DD3010006
:10F4E0000000000031DF010000000000ADC6010097
:10F4F00000000000133025132001320414FFFF1414
:10F5000012010218021928017D12200214400B1862
:10F510006026980425C0EB01144CF10114ECF001B5
:10F520001A44081AF4081A04081AFC081A0C081AD3
:10F5300014041A1C041A24041A2C041A34041A3C45
:08F540000451043C90D00300CB
:040000050001920163
:00000001FF
